Archive member included because of file (symbol)

c:/program files/winavr-20090313/bin/../lib/gcc/avr/4.3.2/avr51\libgcc.a(_mulsi3.o)
                              fat16.o (__mulsi3)
c:/program files/winavr-20090313/bin/../lib/gcc/avr/4.3.2/avr51\libgcc.a(_divmodhi4.o)
                              recording.o (__divmodhi4)
c:/program files/winavr-20090313/bin/../lib/gcc/avr/4.3.2/avr51\libgcc.a(_exit.o)
                              c:/program files/winavr-20090313/bin/../lib/gcc/avr/4.3.2/../../../../avr/lib/avr51/crtm1280.o (exit)
c:/program files/winavr-20090313/bin/../lib/gcc/avr/4.3.2/avr51\libgcc.a(_clear_bss.o)
                              fat16.o (__do_clear_bss)
c:/program files/winavr-20090313/bin/../lib/gcc/avr/4.3.2/avr51\libgcc.a(_mul_sf.o)
                              recording.o (__mulsf3)
c:/program files/winavr-20090313/bin/../lib/gcc/avr/4.3.2/avr51\libgcc.a(_si_to_sf.o)
                              recording.o (__floatsisf)
c:/program files/winavr-20090313/bin/../lib/gcc/avr/4.3.2/avr51\libgcc.a(_sf_to_si.o)
                              recording.o (__fixsfsi)
c:/program files/winavr-20090313/bin/../lib/gcc/avr/4.3.2/avr51\libgcc.a(_thenan_sf.o)
                              c:/program files/winavr-20090313/bin/../lib/gcc/avr/4.3.2/avr51\libgcc.a(_mul_sf.o) (__thenan_sf)
c:/program files/winavr-20090313/bin/../lib/gcc/avr/4.3.2/avr51\libgcc.a(_udivmodhi4.o)
                              c:/program files/winavr-20090313/bin/../lib/gcc/avr/4.3.2/avr51\libgcc.a(_divmodhi4.o) (__udivmodhi4)
c:/program files/winavr-20090313/bin/../lib/gcc/avr/4.3.2/avr51\libgcc.a(_prologue.o)
                              c:/program files/winavr-20090313/bin/../lib/gcc/avr/4.3.2/avr51\libgcc.a(_mul_sf.o) (__prologue_saves__)
c:/program files/winavr-20090313/bin/../lib/gcc/avr/4.3.2/avr51\libgcc.a(_epilogue.o)
                              c:/program files/winavr-20090313/bin/../lib/gcc/avr/4.3.2/avr51\libgcc.a(_mul_sf.o) (__epilogue_restores__)
c:/program files/winavr-20090313/bin/../lib/gcc/avr/4.3.2/avr51\libgcc.a(_clzsi2.o)
                              c:/program files/winavr-20090313/bin/../lib/gcc/avr/4.3.2/avr51\libgcc.a(_si_to_sf.o) (__clzsi2)
c:/program files/winavr-20090313/bin/../lib/gcc/avr/4.3.2/avr51\libgcc.a(_pack_sf.o)
                              c:/program files/winavr-20090313/bin/../lib/gcc/avr/4.3.2/avr51\libgcc.a(_mul_sf.o) (__pack_f)
c:/program files/winavr-20090313/bin/../lib/gcc/avr/4.3.2/avr51\libgcc.a(_unpack_sf.o)
                              c:/program files/winavr-20090313/bin/../lib/gcc/avr/4.3.2/avr51\libgcc.a(_mul_sf.o) (__unpack_f)
c:/program files/winavr-20090313/bin/../lib/gcc/avr/4.3.2/avr51\libgcc.a(_clz.o)
                              c:/program files/winavr-20090313/bin/../lib/gcc/avr/4.3.2/avr51\libgcc.a(_clzsi2.o) (__clz_tab)
c:/program files/winavr-20090313/bin/../lib/gcc/avr/4.3.2/../../../../avr/lib/avr51\libc.a(atoi.o)
                              fat16.o (atoi)
c:/program files/winavr-20090313/bin/../lib/gcc/avr/4.3.2/../../../../avr/lib/avr51\libc.a(strcmp.o)
                              fat16.o (strcmp)
c:/program files/winavr-20090313/bin/../lib/gcc/avr/4.3.2/../../../../avr/lib/avr51\libc.a(strcpy.o)
                              fat16.o (strcpy)
c:/program files/winavr-20090313/bin/../lib/gcc/avr/4.3.2/../../../../avr/lib/avr51\libc.a(strncmp.o)
                              fat16.o (strncmp)
c:/program files/winavr-20090313/bin/../lib/gcc/avr/4.3.2/../../../../avr/lib/avr51\libc.a(itoa.o)
                              fat16.o (itoa)
c:/program files/winavr-20090313/bin/../lib/gcc/avr/4.3.2/../../../../avr/lib/avr51\libc.a(ltoa.o)
                              fat16.o (ltoa)
c:/program files/winavr-20090313/bin/../lib/gcc/avr/4.3.2/../../../../avr/lib/avr51\libc.a(mul10.o)
                              c:/program files/winavr-20090313/bin/../lib/gcc/avr/4.3.2/../../../../avr/lib/avr51\libc.a(atoi.o) (__mulhi_const_10)
c:/program files/winavr-20090313/bin/../lib/gcc/avr/4.3.2/../../../../avr/lib/avr51\libc.a(strrev.o)
                              c:/program files/winavr-20090313/bin/../lib/gcc/avr/4.3.2/../../../../avr/lib/avr51\libc.a(itoa.o) (strrev)
c:/program files/winavr-20090313/bin/../lib/gcc/avr/4.3.2/avr51\libgcc.a(_udivmodsi4.o)
                              c:/program files/winavr-20090313/bin/../lib/gcc/avr/4.3.2/../../../../avr/lib/avr51\libc.a(ltoa.o) (__udivmodsi4)

Allocating common symbols
Common symbol       size              file

fileNameTmp         0x9               recording.o
ACC_Z               0x2               recording.o
BAT                 0x2               recording.o
GYRO_Z45            0x2               recording.o
j                   0x2               fat16.o
SensRecOn           0x1               recording.o
cas                 0x2               ZaznamnikATMEGA1280V1_2_main.o
PresRecOn           0x1               recording.o
pocitadlo           0x4               recording.o
zaznamLimit         0x4               recording.o
ACC_Y               0x2               recording.o
k                   0x2               fat16.o
PRESSURE            0x2               recording.o
debug               0x1               fat16.o
terminalON          0x1               ZaznamnikATMEGA1280V1_2_main.o
buttonDelay         0x1               ZaznamnikATMEGA1280V1_2_main.o
text                0xa               fat16.o
startBlock          0x4               fat16.o
fileEntryNumber     0x2               fat16.o
i                   0x2               fat16.o
SD_ERROR            0x1               recording.o
GyrRecOn            0x1               recording.o
fileEntry           0x1c              fat16.o
data_char           0x1               recording.o
ACC_X               0x2               recording.o
buffer              0x200             ZaznamnikATMEGA1280V1_2_main.o
rootSectorCycle     0x1               fat16.o
totalBlocks         0x4               ZaznamnikATMEGA1280V1_2_main.o
data                0x2               recording.o
fileNumber          0x2               fat16.o
extensionTmp        0x4               recording.o
writeBlockTmp       0x4               fat16.o
dataString          0xa               recording.o
sectorWrittenCount  0x4               fat16.o
bufferWriteInfo     0x4               recording.o
error               0x1               fat16.o
bufferIsFree        0xa               recording.o
GYRO_Y45            0x2               recording.o
rootSector          0x2               fat16.o
FAT_boot            0x3b              fat16.o
AccRecOn            0x1               recording.o
bufferDataGPS       0x2bc             recording.o
bufferData          0x1400            recording.o
GYRO_X45            0x2               recording.o

Memory Configuration

Name             Origin             Length             Attributes
text             0x00000000         0x00020000         xr
data             0x00800060         0x0000ffa0         rw !x
eeprom           0x00810000         0x00010000         rw !x
fuse             0x00820000         0x00000400         rw !x
lock             0x00830000         0x00000400         rw !x
signature        0x00840000         0x00000400         rw !x
*default*        0x00000000         0xffffffff

Linker script and memory map

Address of section .data set to 0x800200
LOAD c:/program files/winavr-20090313/bin/../lib/gcc/avr/4.3.2/../../../../avr/lib/avr51/crtm1280.o
LOAD ADC_ATMEGA1280.o
LOAD fat16.o
LOAD MMA7455L.o
LOAD recording.o
LOAD SD.o
LOAD SPI.o
LOAD UART.o
LOAD ZaznamnikATMEGA1280V1_2_main.o
LOAD c:/program files/winavr-20090313/bin/../lib/gcc/avr/4.3.2/avr51\libgcc.a
LOAD c:/program files/winavr-20090313/bin/../lib/gcc/avr/4.3.2/../../../../avr/lib/avr51\libc.a
LOAD c:/program files/winavr-20090313/bin/../lib/gcc/avr/4.3.2/avr51\libgcc.a

.hash
 *(.hash)

.dynsym
 *(.dynsym)

.dynstr
 *(.dynstr)

.gnu.version
 *(.gnu.version)

.gnu.version_d
 *(.gnu.version_d)

.gnu.version_r
 *(.gnu.version_r)

.rel.init
 *(.rel.init)

.rela.init
 *(.rela.init)

.rel.text
 *(.rel.text)
 *(.rel.text.*)
 *(.rel.gnu.linkonce.t*)

.rela.text
 *(.rela.text)
 *(.rela.text.*)
 *(.rela.gnu.linkonce.t*)

.rel.fini
 *(.rel.fini)

.rela.fini
 *(.rela.fini)

.rel.rodata
 *(.rel.rodata)
 *(.rel.rodata.*)
 *(.rel.gnu.linkonce.r*)

.rela.rodata
 *(.rela.rodata)
 *(.rela.rodata.*)
 *(.rela.gnu.linkonce.r*)

.rel.data
 *(.rel.data)
 *(.rel.data.*)
 *(.rel.gnu.linkonce.d*)

.rela.data
 *(.rela.data)
 *(.rela.data.*)
 *(.rela.gnu.linkonce.d*)

.rel.ctors
 *(.rel.ctors)

.rela.ctors
 *(.rela.ctors)

.rel.dtors
 *(.rel.dtors)

.rela.dtors
 *(.rela.dtors)

.rel.got
 *(.rel.got)

.rela.got
 *(.rela.got)

.rel.bss
 *(.rel.bss)

.rela.bss
 *(.rela.bss)

.rel.plt
 *(.rel.plt)

.rela.plt
 *(.rela.plt)

.text           0x00000000     0x58d6
 *(.vectors)
 .vectors       0x00000000       0xe4 c:/program files/winavr-20090313/bin/../lib/gcc/avr/4.3.2/../../../../avr/lib/avr51/crtm1280.o
                0x00000000                __vectors
                0x00000000                __vector_default
 *(.vectors)
 *(.progmem.gcc*)
 .progmem.gcc_sw_table
                0x000000e4       0x32 ZaznamnikATMEGA1280V1_2_main.o
 *(.progmem*)
 .progmem.data  0x00000116      0x185 fat16.o
 .progmem.data  0x0000029b      0x3fd recording.o
 .progmem.data  0x00000698       0x31 SD.o
 .progmem.data  0x000006c9      0x74d ZaznamnikATMEGA1280V1_2_main.o
                0x00000e16                . = ALIGN (0x2)
                0x00000e16                __trampolines_start = .
 *(.trampolines)
 .trampolines   0x00000e16        0x0 linker stubs
 *(.trampolines*)
                0x00000e16                __trampolines_end = .
 *(.jumptables)
 *(.jumptables*)
 *(.lowtext)
 *(.lowtext*)
                0x00000e16                __ctors_start = .
 *(.ctors)
                0x00000e16                __ctors_end = .
                0x00000e16                __dtors_start = .
 *(.dtors)
                0x00000e16                __dtors_end = .
 SORT(*)(.ctors)
 SORT(*)(.dtors)
 *(.init0)
 .init0         0x00000e16        0x0 c:/program files/winavr-20090313/bin/../lib/gcc/avr/4.3.2/../../../../avr/lib/avr51/crtm1280.o
                0x00000e16                __init
 *(.init0)
 *(.init1)
 *(.init1)
 *(.init2)
 .init2         0x00000e16        0xc c:/program files/winavr-20090313/bin/../lib/gcc/avr/4.3.2/../../../../avr/lib/avr51/crtm1280.o
 *(.init2)
 *(.init3)
 *(.init3)
 *(.init4)
 .init4         0x00000e22       0x1a c:/program files/winavr-20090313/bin/../lib/gcc/avr/4.3.2/../../../../avr/lib/avr51/crtm1280.o
                0x00000e22                __do_copy_data
 .init4         0x00000e3c       0x10 c:/program files/winavr-20090313/bin/../lib/gcc/avr/4.3.2/avr51\libgcc.a(_clear_bss.o)
                0x00000e3c                __do_clear_bss
 *(.init4)
 *(.init5)
 *(.init5)
 *(.init6)
 *(.init6)
 *(.init7)
 *(.init7)
 *(.init8)
 *(.init8)
 *(.init9)
 .init9         0x00000e4c        0x8 c:/program files/winavr-20090313/bin/../lib/gcc/avr/4.3.2/../../../../avr/lib/avr51/crtm1280.o
 *(.init9)
 *(.text)
 .text          0x00000e54        0x4 c:/program files/winavr-20090313/bin/../lib/gcc/avr/4.3.2/../../../../avr/lib/avr51/crtm1280.o
                0x00000e54                __vector_38
                0x00000e54                __vector_22
                0x00000e54                __vector_28
                0x00000e54                __vector_1
                0x00000e54                __vector_32
                0x00000e54                __vector_34
                0x00000e54                __vector_24
                0x00000e54                __vector_12
                0x00000e54                __vector_55
                0x00000e54                __vector_46
                0x00000e54                __bad_interrupt
                0x00000e54                __vector_6
                0x00000e54                __vector_31
                0x00000e54                __vector_39
                0x00000e54                __vector_3
                0x00000e54                __vector_23
                0x00000e54                __vector_30
                0x00000e54                __vector_25
                0x00000e54                __vector_11
                0x00000e54                __vector_13
                0x00000e54                __vector_17
                0x00000e54                __vector_19
                0x00000e54                __vector_56
                0x00000e54                __vector_7
                0x00000e54                __vector_49
                0x00000e54                __vector_41
                0x00000e54                __vector_43
                0x00000e54                __vector_27
                0x00000e54                __vector_5
                0x00000e54                __vector_33
                0x00000e54                __vector_52
                0x00000e54                __vector_37
                0x00000e54                __vector_4
                0x00000e54                __vector_44
                0x00000e54                __vector_51
                0x00000e54                __vector_9
                0x00000e54                __vector_2
                0x00000e54                __vector_21
                0x00000e54                __vector_15
                0x00000e54                __vector_29
                0x00000e54                __vector_40
                0x00000e54                __vector_8
                0x00000e54                __vector_26
                0x00000e54                __vector_14
                0x00000e54                __vector_53
                0x00000e54                __vector_10
                0x00000e54                __vector_16
                0x00000e54                __vector_18
                0x00000e54                __vector_20
                0x00000e54                __vector_42
 .text          0x00000e58       0x40 ADC_ATMEGA1280.o
                0x00000e78                ADConversion
                0x00000e58                ADCinit
 .text          0x00000e98     0x1bdc fat16.o
                0x0000224a                readFile
                0x00002458                getNextFreeFileIndexNumber
                0x00001964                appendOpenedFile
                0x000017d8                fileList
                0x00000e98                findFreeCluster
                0x00001018                findNextCluster
                0x00001fea                findFile
                0x000010e8                closeOpenedFile
                0x0000275e                openNewFile
                0x00001490                readFatBoot
                0x00001db6                fatInfo
 .text          0x00002a74      0x210 MMA7455L.o
                0x00002b96                accReadRegister
                0x00002a74                accWriteRegister
                0x00002b78                accInit
 .text          0x00002c84     0x1088 recording.o
                0x000037c6                recordingStart
                0x00003682                stav
                0x0000327a                __vector_35
                0x00002efc                uvozovaciVetaBufferWrite
                0x00002d00                __vector_45
                0x00002c86                __vector_54
                0x000039f0                test
                0x00002df0                __vector_47
                0x00002fc6                endOfLineBufferWrite
                0x0000315a                commaBufferWrite
                0x00002e28                dataStringBufferWrite
                0x00003090                numberSpaceBufferWrite
                0x000031ea                startOfLineBufferWrite
                0x00002e12                __vector_48
                0x00002dbc                __vector_50
                0x00002c84                test_c
 .text          0x00003d0c      0x5f4 SD.o
                0x00003d72                SD_erase
                0x000041e6                SD_writeSingleBlock
                0x0000404a                SD_readMultipleBlock
                0x00003d0c                SD_sendCommand
                0x00004126                SD_writeSingleBlockData
                0x00004290                SD_readSingleBlock
                0x00003e8c                SD_writeMultipleBlock
                0x00003df4                SD_init
 .text          0x00004300       0x28 SPI.o
                0x0000430e                SPI_transmit
                0x00004300                spi_init
                0x0000431a                SPI_receive
 .text          0x00004328       0x78 UART.o
                0x0000436c                transmitString_FUART1
                0x0000433a                receiveByteUART3
                0x00004386                transmitStringUART1
                0x0000435c                transmitByteUART2
                0x0000434c                transmitByteUART1
                0x00004328                receiveByteUART1
 .text          0x000043a0      0xc12 ZaznamnikATMEGA1280V1_2_main.o
                0x000043a0                port_init
                0x0000444a                del
                0x00004414                timer5_init
                0x000043a8                uart1_init
                0x00004522                led_vyp
                0x00004470                GPS_config
                0x000043cc                uart1_off
                0x000043f6                timer3_init
                0x000048ce                test_b
                0x00004a7a                main
                0x000046e0                shblk
                0x0000444e                soub_zap
                0x0000454a                help
                0x00004a74                dir
                0x00004450                __vector_36
                0x000043d2                uart3_init
                0x0000444c                wrblk
                0x000048d8                soub_zobr
 .text          0x00004fb2        0x0 c:/program files/winavr-20090313/bin/../lib/gcc/avr/4.3.2/avr51\libgcc.a(_mulsi3.o)
 .text          0x00004fb2        0x0 c:/program files/winavr-20090313/bin/../lib/gcc/avr/4.3.2/avr51\libgcc.a(_divmodhi4.o)
 .text          0x00004fb2        0x0 c:/program files/winavr-20090313/bin/../lib/gcc/avr/4.3.2/avr51\libgcc.a(_exit.o)
 .text          0x00004fb2        0x0 c:/program files/winavr-20090313/bin/../lib/gcc/avr/4.3.2/avr51\libgcc.a(_clear_bss.o)
 .text          0x00004fb2      0x1f4 c:/program files/winavr-20090313/bin/../lib/gcc/avr/4.3.2/avr51\libgcc.a(_mul_sf.o)
                0x00004fb2                __mulsf3
 .text          0x000051a6       0xbc c:/program files/winavr-20090313/bin/../lib/gcc/avr/4.3.2/avr51\libgcc.a(_si_to_sf.o)
                0x000051a6                __floatsisf
 .text          0x00005262       0xa8 c:/program files/winavr-20090313/bin/../lib/gcc/avr/4.3.2/avr51\libgcc.a(_sf_to_si.o)
                0x00005262                __fixsfsi
 .text          0x0000530a        0x0 c:/program files/winavr-20090313/bin/../lib/gcc/avr/4.3.2/avr51\libgcc.a(_thenan_sf.o)
 .text          0x0000530a        0x0 c:/program files/winavr-20090313/bin/../lib/gcc/avr/4.3.2/avr51\libgcc.a(_udivmodhi4.o)
 .text          0x0000530a        0x0 c:/program files/winavr-20090313/bin/../lib/gcc/avr/4.3.2/avr51\libgcc.a(_prologue.o)
 .text          0x0000530a        0x0 c:/program files/winavr-20090313/bin/../lib/gcc/avr/4.3.2/avr51\libgcc.a(_epilogue.o)
 .text          0x0000530a       0x9e c:/program files/winavr-20090313/bin/../lib/gcc/avr/4.3.2/avr51\libgcc.a(_clzsi2.o)
                0x0000530a                __clzsi2
 .text          0x000053a8      0x1aa c:/program files/winavr-20090313/bin/../lib/gcc/avr/4.3.2/avr51\libgcc.a(_pack_sf.o)
                0x000053a8                __pack_f
 .text          0x00005552       0xf0 c:/program files/winavr-20090313/bin/../lib/gcc/avr/4.3.2/avr51\libgcc.a(_unpack_sf.o)
                0x00005552                __unpack_f
 .text          0x00005642        0x0 c:/program files/winavr-20090313/bin/../lib/gcc/avr/4.3.2/avr51\libgcc.a(_clz.o)
 .text          0x00005642       0x3c c:/program files/winavr-20090313/bin/../lib/gcc/avr/4.3.2/../../../../avr/lib/avr51\libc.a(atoi.o)
                0x00005642                atoi
 .text          0x0000567e       0x12 c:/program files/winavr-20090313/bin/../lib/gcc/avr/4.3.2/../../../../avr/lib/avr51\libc.a(strcmp.o)
                0x0000567e                strcmp
 .text          0x00005690        0xe c:/program files/winavr-20090313/bin/../lib/gcc/avr/4.3.2/../../../../avr/lib/avr51\libc.a(strcpy.o)
                0x00005690                strcpy
 .text          0x0000569e       0x1c c:/program files/winavr-20090313/bin/../lib/gcc/avr/4.3.2/../../../../avr/lib/avr51\libc.a(strncmp.o)
                0x0000569e                strncmp
 .text          0x000056ba       0x42 c:/program files/winavr-20090313/bin/../lib/gcc/avr/4.3.2/../../../../avr/lib/avr51\libc.a(itoa.o)
                0x000056ba                itoa
 .text          0x000056fc       0x68 c:/program files/winavr-20090313/bin/../lib/gcc/avr/4.3.2/../../../../avr/lib/avr51\libc.a(ltoa.o)
                0x000056fc                ltoa
 .text          0x00005764       0x10 c:/program files/winavr-20090313/bin/../lib/gcc/avr/4.3.2/../../../../avr/lib/avr51\libc.a(mul10.o)
                0x00005764                __mulhi_const_10
 .text          0x00005774       0x20 c:/program files/winavr-20090313/bin/../lib/gcc/avr/4.3.2/../../../../avr/lib/avr51\libc.a(strrev.o)
                0x00005774                strrev
 .text          0x00005794        0x0 c:/program files/winavr-20090313/bin/../lib/gcc/avr/4.3.2/avr51\libgcc.a(_udivmodsi4.o)
                0x00005794                . = ALIGN (0x2)
 *(.text.*)
 .text.libgcc   0x00005794       0x3e c:/program files/winavr-20090313/bin/../lib/gcc/avr/4.3.2/avr51\libgcc.a(_mulsi3.o)
                0x00005794                __mulsi3
 .text.libgcc   0x000057d2       0x26 c:/program files/winavr-20090313/bin/../lib/gcc/avr/4.3.2/avr51\libgcc.a(_divmodhi4.o)
                0x000057d2                __divmodhi4
                0x000057d2                _div
 .text.libgcc   0x000057f8        0x0 c:/program files/winavr-20090313/bin/../lib/gcc/avr/4.3.2/avr51\libgcc.a(_exit.o)
 .text.libgcc   0x000057f8        0x0 c:/program files/winavr-20090313/bin/../lib/gcc/avr/4.3.2/avr51\libgcc.a(_clear_bss.o)
 .text.libgcc   0x000057f8       0x28 c:/program files/winavr-20090313/bin/../lib/gcc/avr/4.3.2/avr51\libgcc.a(_udivmodhi4.o)
                0x000057f8                __udivmodhi4
 .text.libgcc   0x00005820       0x38 c:/program files/winavr-20090313/bin/../lib/gcc/avr/4.3.2/avr51\libgcc.a(_prologue.o)
                0x00005820                __prologue_saves__
 .text.libgcc   0x00005858       0x36 c:/program files/winavr-20090313/bin/../lib/gcc/avr/4.3.2/avr51\libgcc.a(_epilogue.o)
                0x00005858                __epilogue_restores__
 .text.libgcc   0x0000588e       0x44 c:/program files/winavr-20090313/bin/../lib/gcc/avr/4.3.2/avr51\libgcc.a(_udivmodsi4.o)
                0x0000588e                __udivmodsi4
                0x000058d2                . = ALIGN (0x2)
 *(.fini9)
 .fini9         0x000058d2        0x0 c:/program files/winavr-20090313/bin/../lib/gcc/avr/4.3.2/avr51\libgcc.a(_exit.o)
                0x000058d2                exit
                0x000058d2                _exit
 *(.fini9)
 *(.fini8)
 *(.fini8)
 *(.fini7)
 *(.fini7)
 *(.fini6)
 *(.fini6)
 *(.fini5)
 *(.fini5)
 *(.fini4)
 *(.fini4)
 *(.fini3)
 *(.fini3)
 *(.fini2)
 *(.fini2)
 *(.fini1)
 *(.fini1)
 *(.fini0)
 .fini0         0x000058d2        0x4 c:/program files/winavr-20090313/bin/../lib/gcc/avr/4.3.2/avr51\libgcc.a(_exit.o)
 *(.fini0)
                0x000058d6                _etext = .

.data           0x00800200      0x150 load address 0x000058d6
                0x00800200                PROVIDE (__data_start, .)
 *(.data)
 .data          0x00800200        0x0 c:/program files/winavr-20090313/bin/../lib/gcc/avr/4.3.2/../../../../avr/lib/avr51/crtm1280.o
 .data          0x00800200        0x0 ADC_ATMEGA1280.o
 .data          0x00800200        0x0 fat16.o
 .data          0x00800200        0x0 MMA7455L.o
 .data          0x00800200       0x11 recording.o
                0x0080020d                ADconst
 .data          0x00800211        0x0 SD.o
 .data          0x00800211        0x0 SPI.o
 .data          0x00800211        0x0 UART.o
 .data          0x00800211       0x37 ZaznamnikATMEGA1280V1_2_main.o
 .data          0x00800248        0x0 c:/program files/winavr-20090313/bin/../lib/gcc/avr/4.3.2/avr51\libgcc.a(_mulsi3.o)
 .data          0x00800248        0x0 c:/program files/winavr-20090313/bin/../lib/gcc/avr/4.3.2/avr51\libgcc.a(_divmodhi4.o)
 .data          0x00800248        0x0 c:/program files/winavr-20090313/bin/../lib/gcc/avr/4.3.2/avr51\libgcc.a(_exit.o)
 .data          0x00800248        0x0 c:/program files/winavr-20090313/bin/../lib/gcc/avr/4.3.2/avr51\libgcc.a(_clear_bss.o)
 .data          0x00800248        0x0 c:/program files/winavr-20090313/bin/../lib/gcc/avr/4.3.2/avr51\libgcc.a(_mul_sf.o)
 .data          0x00800248        0x0 c:/program files/winavr-20090313/bin/../lib/gcc/avr/4.3.2/avr51\libgcc.a(_si_to_sf.o)
 .data          0x00800248        0x0 c:/program files/winavr-20090313/bin/../lib/gcc/avr/4.3.2/avr51\libgcc.a(_sf_to_si.o)
 .data          0x00800248        0x8 c:/program files/winavr-20090313/bin/../lib/gcc/avr/4.3.2/avr51\libgcc.a(_thenan_sf.o)
                0x00800248                __thenan_sf
 .data          0x00800250        0x0 c:/program files/winavr-20090313/bin/../lib/gcc/avr/4.3.2/avr51\libgcc.a(_udivmodhi4.o)
 .data          0x00800250        0x0 c:/program files/winavr-20090313/bin/../lib/gcc/avr/4.3.2/avr51\libgcc.a(_prologue.o)
 .data          0x00800250        0x0 c:/program files/winavr-20090313/bin/../lib/gcc/avr/4.3.2/avr51\libgcc.a(_epilogue.o)
 .data          0x00800250        0x0 c:/program files/winavr-20090313/bin/../lib/gcc/avr/4.3.2/avr51\libgcc.a(_clzsi2.o)
 .data          0x00800250        0x0 c:/program files/winavr-20090313/bin/../lib/gcc/avr/4.3.2/avr51\libgcc.a(_pack_sf.o)
 .data          0x00800250        0x0 c:/program files/winavr-20090313/bin/../lib/gcc/avr/4.3.2/avr51\libgcc.a(_unpack_sf.o)
 .data          0x00800250      0x100 c:/program files/winavr-20090313/bin/../lib/gcc/avr/4.3.2/avr51\libgcc.a(_clz.o)
                0x00800250                __clz_tab
 .data          0x00800350        0x0 c:/program files/winavr-20090313/bin/../lib/gcc/avr/4.3.2/../../../../avr/lib/avr51\libc.a(atoi.o)
 .data          0x00800350        0x0 c:/program files/winavr-20090313/bin/../lib/gcc/avr/4.3.2/../../../../avr/lib/avr51\libc.a(strcmp.o)
 .data          0x00800350        0x0 c:/program files/winavr-20090313/bin/../lib/gcc/avr/4.3.2/../../../../avr/lib/avr51\libc.a(strcpy.o)
 .data          0x00800350        0x0 c:/program files/winavr-20090313/bin/../lib/gcc/avr/4.3.2/../../../../avr/lib/avr51\libc.a(strncmp.o)
 .data          0x00800350        0x0 c:/program files/winavr-20090313/bin/../lib/gcc/avr/4.3.2/../../../../avr/lib/avr51\libc.a(itoa.o)
 .data          0x00800350        0x0 c:/program files/winavr-20090313/bin/../lib/gcc/avr/4.3.2/../../../../avr/lib/avr51\libc.a(ltoa.o)
 .data          0x00800350        0x0 c:/program files/winavr-20090313/bin/../lib/gcc/avr/4.3.2/../../../../avr/lib/avr51\libc.a(mul10.o)
 .data          0x00800350        0x0 c:/program files/winavr-20090313/bin/../lib/gcc/avr/4.3.2/../../../../avr/lib/avr51\libc.a(strrev.o)
 .data          0x00800350        0x0 c:/program files/winavr-20090313/bin/../lib/gcc/avr/4.3.2/avr51\libgcc.a(_udivmodsi4.o)
 *(.data*)
 *(.rodata)
 *(.rodata*)
 *(.gnu.linkonce.d*)
                0x00800350                . = ALIGN (0x2)
                0x00800350                _edata = .
                0x00800350                PROVIDE (__data_end, .)

.bss            0x00800350     0x1997
                0x00800350                PROVIDE (__bss_start, .)
 *(.bss)
 .bss           0x00800350        0x0 c:/program files/winavr-20090313/bin/../lib/gcc/avr/4.3.2/../../../../avr/lib/avr51/crtm1280.o
 .bss           0x00800350        0x0 ADC_ATMEGA1280.o
 .bss           0x00800350        0x0 fat16.o
 .bss           0x00800350        0x0 MMA7455L.o
 .bss           0x00800350       0x11 recording.o
                0x00800355                zapis
                0x00800352                led1isON
                0x00800353                led3isON
                0x00800350                batCycleDivider
                0x00800354                GPS_FIX
                0x0080035a                gpsBuf
                0x00800358                buf
                0x0080035c                whil
                0x00800360                bufferWriteSD
                0x0080035f                bufferWrite
                0x0080035e                bufferDataGPSFull
                0x00800357                zaznamSpusten
 .bss           0x00800361        0x0 SD.o
 .bss           0x00800361        0x0 SPI.o
 .bss           0x00800361        0x0 UART.o
 .bss           0x00800361        0x1 ZaznamnikATMEGA1280V1_2_main.o
                0x00800361                gpsOutputON
 .bss           0x00800362        0x0 c:/program files/winavr-20090313/bin/../lib/gcc/avr/4.3.2/avr51\libgcc.a(_mulsi3.o)
 .bss           0x00800362        0x0 c:/program files/winavr-20090313/bin/../lib/gcc/avr/4.3.2/avr51\libgcc.a(_divmodhi4.o)
 .bss           0x00800362        0x0 c:/program files/winavr-20090313/bin/../lib/gcc/avr/4.3.2/avr51\libgcc.a(_exit.o)
 .bss           0x00800362        0x0 c:/program files/winavr-20090313/bin/../lib/gcc/avr/4.3.2/avr51\libgcc.a(_clear_bss.o)
 .bss           0x00800362        0x0 c:/program files/winavr-20090313/bin/../lib/gcc/avr/4.3.2/avr51\libgcc.a(_mul_sf.o)
 .bss           0x00800362        0x0 c:/program files/winavr-20090313/bin/../lib/gcc/avr/4.3.2/avr51\libgcc.a(_si_to_sf.o)
 .bss           0x00800362        0x0 c:/program files/winavr-20090313/bin/../lib/gcc/avr/4.3.2/avr51\libgcc.a(_sf_to_si.o)
 .bss           0x00800362        0x0 c:/program files/winavr-20090313/bin/../lib/gcc/avr/4.3.2/avr51\libgcc.a(_thenan_sf.o)
 .bss           0x00800362        0x0 c:/program files/winavr-20090313/bin/../lib/gcc/avr/4.3.2/avr51\libgcc.a(_udivmodhi4.o)
 .bss           0x00800362        0x0 c:/program files/winavr-20090313/bin/../lib/gcc/avr/4.3.2/avr51\libgcc.a(_prologue.o)
 .bss           0x00800362        0x0 c:/program files/winavr-20090313/bin/../lib/gcc/avr/4.3.2/avr51\libgcc.a(_epilogue.o)
 .bss           0x00800362        0x0 c:/program files/winavr-20090313/bin/../lib/gcc/avr/4.3.2/avr51\libgcc.a(_clzsi2.o)
 .bss           0x00800362        0x0 c:/program files/winavr-20090313/bin/../lib/gcc/avr/4.3.2/avr51\libgcc.a(_pack_sf.o)
 .bss           0x00800362        0x0 c:/program files/winavr-20090313/bin/../lib/gcc/avr/4.3.2/avr51\libgcc.a(_unpack_sf.o)
 .bss           0x00800362        0x0 c:/program files/winavr-20090313/bin/../lib/gcc/avr/4.3.2/avr51\libgcc.a(_clz.o)
 .bss           0x00800362        0x0 c:/program files/winavr-20090313/bin/../lib/gcc/avr/4.3.2/../../../../avr/lib/avr51\libc.a(atoi.o)
 .bss           0x00800362        0x0 c:/program files/winavr-20090313/bin/../lib/gcc/avr/4.3.2/../../../../avr/lib/avr51\libc.a(strcmp.o)
 .bss           0x00800362        0x0 c:/program files/winavr-20090313/bin/../lib/gcc/avr/4.3.2/../../../../avr/lib/avr51\libc.a(strcpy.o)
 .bss           0x00800362        0x0 c:/program files/winavr-20090313/bin/../lib/gcc/avr/4.3.2/../../../../avr/lib/avr51\libc.a(strncmp.o)
 .bss           0x00800362        0x0 c:/program files/winavr-20090313/bin/../lib/gcc/avr/4.3.2/../../../../avr/lib/avr51\libc.a(itoa.o)
 .bss           0x00800362        0x0 c:/program files/winavr-20090313/bin/../lib/gcc/avr/4.3.2/../../../../avr/lib/avr51\libc.a(ltoa.o)
 .bss           0x00800362        0x0 c:/program files/winavr-20090313/bin/../lib/gcc/avr/4.3.2/../../../../avr/lib/avr51\libc.a(mul10.o)
 .bss           0x00800362        0x0 c:/program files/winavr-20090313/bin/../lib/gcc/avr/4.3.2/../../../../avr/lib/avr51\libc.a(strrev.o)
 .bss           0x00800362        0x0 c:/program files/winavr-20090313/bin/../lib/gcc/avr/4.3.2/avr51\libgcc.a(_udivmodsi4.o)
 *(.bss*)
 *(COMMON)
 COMMON         0x00800362       0x7c fat16.o
                0x00800362                j
                0x00800364                k
                0x00800366                debug
                0x00800367                text
                0x00800371                startBlock
                0x00800375                fileEntryNumber
                0x00800377                i
                0x00800379                fileEntry
                0x00800395                rootSectorCycle
                0x00800396                fileNumber
                0x00800398                writeBlockTmp
                0x0080039c                sectorWrittenCount
                0x008003a0                error
                0x008003a1                rootSector
                0x008003a3                FAT_boot
 COMMON         0x008003de     0x1701 recording.o
                0x008003de                fileNameTmp
                0x008003e7                ACC_Z
                0x008003e9                BAT
                0x008003eb                GYRO_Z45
                0x008003ed                SensRecOn
                0x008003ee                PresRecOn
                0x008003ef                pocitadlo
                0x008003f3                zaznamLimit
                0x008003f7                ACC_Y
                0x008003f9                PRESSURE
                0x008003fb                SD_ERROR
                0x008003fc                GyrRecOn
                0x008003fd                data_char
                0x008003fe                ACC_X
                0x00800400                data
                0x00800402                extensionTmp
                0x00800406                dataString
                0x00800410                bufferWriteInfo
                0x00800414                bufferIsFree
                0x0080041e                GYRO_Y45
                0x00800420                AccRecOn
                0x00800421                bufferDataGPS
                0x008006dd                bufferData
                0x00801add                GYRO_X45
 COMMON         0x00801adf      0x208 ZaznamnikATMEGA1280V1_2_main.o
                0x00801adf                cas
                0x00801ae1                terminalON
                0x00801ae2                buttonDelay
                0x00801ae3                buffer
                0x00801ce3                totalBlocks
                0x00801ce7                PROVIDE (__bss_end, .)
                0x000058d6                __data_load_start = LOADADDR (.data)
                0x00005a26                __data_load_end = (__data_load_start + SIZEOF (.data))

.noinit         0x00801ce7        0x0
                0x00801ce7                PROVIDE (__noinit_start, .)
 *(.noinit*)
                0x00801ce7                PROVIDE (__noinit_end, .)
                0x00801ce7                _end = .
                0x00801ce7                PROVIDE (__heap_start, .)

.eeprom         0x00810000        0x0
 *(.eeprom*)
                0x00810000                __eeprom_end = .

.fuse
 *(.fuse)
 *(.lfuse)
 *(.hfuse)
 *(.efuse)

.lock
 *(.lock*)

.signature
 *(.signature*)

.stab
 *(.stab)

.stabstr
 *(.stabstr)

.stab.excl
 *(.stab.excl)

.stab.exclstr
 *(.stab.exclstr)

.stab.index
 *(.stab.index)

.stab.indexstr
 *(.stab.indexstr)

.comment
 *(.comment)

.debug
 *(.debug)

.line
 *(.line)

.debug_srcinfo
 *(.debug_srcinfo)

.debug_sfnames
 *(.debug_sfnames)

.debug_aranges  0x00000000      0x100
 *(.debug_aranges)
 .debug_aranges
                0x00000000       0x20 ADC_ATMEGA1280.o
 .debug_aranges
                0x00000020       0x20 fat16.o
 .debug_aranges
                0x00000040       0x20 MMA7455L.o
 .debug_aranges
                0x00000060       0x20 recording.o
 .debug_aranges
                0x00000080       0x20 SD.o
 .debug_aranges
                0x000000a0       0x20 SPI.o
 .debug_aranges
                0x000000c0       0x20 UART.o
 .debug_aranges
                0x000000e0       0x20 ZaznamnikATMEGA1280V1_2_main.o

.debug_pubnames
                0x00000000      0x8db
 *(.debug_pubnames)
 .debug_pubnames
                0x00000000       0x2f ADC_ATMEGA1280.o
 .debug_pubnames
                0x0000002f      0x19d fat16.o
 .debug_pubnames
                0x000001cc       0x47 MMA7455L.o
 .debug_pubnames
                0x00000213      0x34f recording.o
 .debug_pubnames
                0x00000562       0xbc SD.o
 .debug_pubnames
                0x0000061e       0x40 SPI.o
 .debug_pubnames
                0x0000065e       0x9a UART.o
 .debug_pubnames
                0x000006f8      0x1e3 ZaznamnikATMEGA1280V1_2_main.o

.debug_info     0x00000000     0x323d
 *(.debug_info)
 .debug_info    0x00000000       0x96 ADC_ATMEGA1280.o
 .debug_info    0x00000096      0x824 fat16.o
 .debug_info    0x000008ba      0x398 MMA7455L.o
 .debug_info    0x00000c52      0xcad recording.o
 .debug_info    0x000018ff      0x3f9 SD.o
 .debug_info    0x00001cf8       0xc6 SPI.o
 .debug_info    0x00001dbe      0x21c UART.o
 .debug_info    0x00001fda     0x1263 ZaznamnikATMEGA1280V1_2_main.o
 *(.gnu.linkonce.wi.*)

.debug_abbrev   0x00000000      0xaea
 *(.debug_abbrev)
 .debug_abbrev  0x00000000       0x63 ADC_ATMEGA1280.o
 .debug_abbrev  0x00000063      0x1d4 fat16.o
 .debug_abbrev  0x00000237      0x153 MMA7455L.o
 .debug_abbrev  0x0000038a      0x219 recording.o
 .debug_abbrev  0x000005a3      0x149 SD.o
 .debug_abbrev  0x000006ec       0x8d SPI.o
 .debug_abbrev  0x00000779      0x122 UART.o
 .debug_abbrev  0x0000089b      0x24f ZaznamnikATMEGA1280V1_2_main.o

.debug_line     0x00000000     0x30c9
 *(.debug_line)
 .debug_line    0x00000000       0xb8 ADC_ATMEGA1280.o
 .debug_line    0x000000b8      0xa7c fat16.o
 .debug_line    0x00000b34      0x32f MMA7455L.o
 .debug_line    0x00000e63      0xbea recording.o
 .debug_line    0x00001a4d      0x592 SD.o
 .debug_line    0x00001fdf       0xcd SPI.o
 .debug_line    0x000020ac      0x18d UART.o
 .debug_line    0x00002239      0xe90 ZaznamnikATMEGA1280V1_2_main.o

.debug_frame    0x00000000      0x4b0
 *(.debug_frame)
 .debug_frame   0x00000000       0x30 ADC_ATMEGA1280.o
 .debug_frame   0x00000030       0xc0 fat16.o
 .debug_frame   0x000000f0       0x40 MMA7455L.o
 .debug_frame   0x00000130      0x110 recording.o
 .debug_frame   0x00000240       0x90 SD.o
 .debug_frame   0x000002d0       0x40 SPI.o
 .debug_frame   0x00000310       0x70 UART.o
 .debug_frame   0x00000380      0x130 ZaznamnikATMEGA1280V1_2_main.o

.debug_str      0x00000000      0xa88
 *(.debug_str)
 .debug_str     0x00000000       0xbf ADC_ATMEGA1280.o
                                 0xf3 (size before relaxing)
 .debug_str     0x000000bf      0x332 fat16.o
                                0x3f8 (size before relaxing)
 .debug_str     0x000003f1       0x93 MMA7455L.o
                                0x16a (size before relaxing)
 .debug_str     0x00000484      0x2bc recording.o
                                0x3e9 (size before relaxing)
 .debug_str     0x00000740       0xc9 SD.o
                                0x1a6 (size before relaxing)
 .debug_str     0x00000809       0x2b SPI.o
                                 0xf1 (size before relaxing)
 .debug_str     0x00000834       0x88 UART.o
                                0x176 (size before relaxing)
 .debug_str     0x000008bc      0x1cc ZaznamnikATMEGA1280V1_2_main.o
                                0x387 (size before relaxing)

.debug_loc      0x00000000     0x122e
 *(.debug_loc)
 .debug_loc     0x00000000      0x2d4 fat16.o
 .debug_loc     0x000002d4      0x120 MMA7455L.o
 .debug_loc     0x000003f4      0x1d8 recording.o
 .debug_loc     0x000005cc      0x602 SD.o
 .debug_loc     0x00000bce       0x26 SPI.o
 .debug_loc     0x00000bf4       0xd8 UART.o
 .debug_loc     0x00000ccc      0x562 ZaznamnikATMEGA1280V1_2_main.o

.debug_macinfo
 *(.debug_macinfo)
OUTPUT(ZaznamnikATMEGA1280V1_2.elf elf32-avr)
LOAD linker stubs

.debug_ranges   0x00000000      0x288
 .debug_ranges  0x00000000      0x180 MMA7455L.o
 .debug_ranges  0x00000180       0x48 recording.o
 .debug_ranges  0x000001c8       0x30 UART.o
 .debug_ranges  0x000001f8       0x90 ZaznamnikATMEGA1280V1_2_main.o
